:020000040000FA
:04080000E4EF04F02D
:1008100003B23DEF04F0F2B458EF04F09EB060EF85
:1008200004F09EB268EF04F0F2A81AEF04F0F2B2FE
:100830001CEF04F0C2EF04F0CD90F29207BC078EDB
:10084000078C9EA029EF04F00101463F29EF04F038
:10085000472B07AE34EF04F0CECF4EF1CFCF4FF1A0
:1008600046C150F147C151F1CF6ACE6A0101466BD2
:10087000476B9E90CD80C2EF04F00392030103EE1C
:1008800000F080517F0BE92604C0EFFF802B8151DF
:10089000805D700BD8A48B8200008051815D700B4D
:1008A000D8A48B9281518019D8B40790C2EF04F07C
:1008B000F2940101383FC2EF04F0392BC2EF04F08B
:1008C0009E900101463FC2EF04F0472BC2EF04F0B7
:1008D0009E92C3CF48F1C4CF49F1C28207B485EFDD
:1008E00004F0220E3E6F000E3F6F000E406F000EB0
:1008F000416F000E526F100E536F0E0E546F000EAC
:10090000556FE30E4A6F000E4B6F0201002FC2EFCE
:1009100004F03C0E006FD57ED5BE32D0D6CF3AF172
:10092000D7CF3BF138C13CF1E86AE8CF3DF1010196
:1009300047A7A6EF04F0079C079E0101000E4E6F2B
:10094000600E4F6F3D0E506F080E516F01013ABFA0
:10095000B6EF04F03B67B6EF04F03C67B6EF04F087
:100960003D67B6EF04F0F288BBEF04F0F2984E6BEF
:100970004F6B506B516BD76AD66A0101386B396B7C
:10098000C2EF04F002C0E0FF005001C0D8FF100029
:10099000A6B2C8EF04F00CC0A9FF0BC0A8FFA69E2A
:1009A000A69CA684F29E550EA76EAA0EA76EA682DE
:1009B000F28EA694A6B2DAEF04F01200A96EA69EFB
:1009C000A69CA680A85012000F010E0EC16E800ECC
:1009D000C06E030EC26E0F01896A110E926E080E70
:1009E0008A6EF10E936E8B6A800E946EF18E0F01FB
:1009F000280ED56EF28AB00ECD6E9D8001014E6B31
:100A00004F6B506B516B526B536B546B556B566BFA
:100A1000576B586B596B079C079E760ECA6E9D826A
:100A200002013C0E006FCC6A240EAC6E0401806B98
:100A3000816B0F01900EAB6E0F019D8A0301806BDD
:100A4000816B8A6B8B920001F28EF28C07B0EAEF19
:100A50000AF00301805181197F0BD8B4EAEF0AF044
:100A600013EE00F081517F0BE126812BE7CFE8FFE9
:100A7000E00BD8B4EAEF0AF023EE82F08A51070BBC
:100A8000D926E7CFDFFF8A2BDF50780AD8A4EAEF18
:100A90000AF007808251720AD8B4ECEF06F0825156
:100AA000630AD8B42CEF09F08251690AD8B473EF05
:100AB00005F082517A0AD8B486EF06F061EF09F0AA
:100AC000040114EE00F080517F0BE12682C4E7FFA1
:100AD000802B12000D0E826F60EC05F00A0E826F03
:100AE00060EC05F012000401690E826F60EC05F005
:100AF00004012C0E826F60EC05F00101030E006F03
:100B0000000E016F000E026F000E036F8DEC0DF0F2
:100B100020C182F40401300E822760EC05F021C16F
:100B200082F40401300E822760EC05F022C182F4C9
:100B30000401300E822760EC05F023C182F4040129
:100B4000300E822760EC05F024C182F40401300EDF
:100B5000822760EC05F025C182F40401300E822763
:100B600060EC05F026C182F40401300E822760ECAF
:100B700005F027C182F40401300E822760EC05F0F5
:100B800004012C0E826F60EC05F00101030E006F72
:100B9000000E016F000E026F000E036F8DEC0DF062
:100BA00020C182F40401300E822760EC05F021C1DF
:100BB00082F40401300E822760EC05F022C182F439
:100BC0000401300E822760EC05F023C182F4040199
:100BD000300E822760EC05F024C182F40401300E4F
:100BE000822760EC05F025C182F40401300E8227D3
:100BF00060EC05F026C182F40401300E822760EC1F
:100C000005F027C182F40401300E822760EC05F064
:100C100004012C0E826F60EC05F00101080E006FDC
:100C2000000E016F000E026F000E036F8DEC0DF0D1
:100C300020C182F40401300E822760EC05F021C14E
:100C400082F40401300E822760EC05F022C182F4A8
:100C50000401300E822760EC05F023C182F4040108
:100C6000300E822760EC05F024C182F40401300EBE
:100C7000822760EC05F025C182F40401300E822742
:100C800060EC05F026C182F40401300E822760EC8E
:100C900005F027C182F40401300E822760EC05F0D4
:100CA00004012C0E826F60EC05F0200EF86EF76ADE
:100CB000F66A04010900F5CF82F460EC05F0090042
:100CC000F5CF82F460EC05F00900F5CF82F460EC1A
:100CD00005F00900F5CF82F460EC05F00900F5CFCE
:100CE00082F460EC05F00900F5CF82F460EC05F0C9
:100CF0000900F5CF82F460EC05F00900F5CF82F42D
:100D000060EC05F06AEC05F061EF09F08351630ACD
:100D1000D8A461EF09F08451610AD8A461EF09F009
:100D200085516C0AD8A461EF09F08651410A2EE082
:100D30008651440A07E08651420AD8B4D9EF06F03A
:100D400061EF09F00798079A04017A0E826F60EC50
:100D500005F00401780E826F60EC05F00401640E6A
:100D6000826F60EC05F081A8BDEF06F00401550E1E
:100D7000826F60EC05F0C2EF06F004014C0E826F4A
:100D800060EC05F06AEC05F061EF09F00788079A5E
:100D900004017A0E826F60EC05F00401410E826F4F
:100DA00060EC05F00401610E826F60EC05F0B3EFBA
:100DB00006F00798078A04017A0E826F60EC05F04E
:100DC0000401420E826F60EC05F00401610E826F37
:100DD00060EC05F0B3EF06F00401720E826F60EC78
:100DE00005F004012C0E826F60EC05F0078452C1FF
:100DF00056F153C157F154C158F155C159F13EC193
:100E000042F13FC143F140C144F141C145F14AC102
:100E10004CF14BC14DF107940101620E046F010EBC
:100E2000056F000E066F000E076F56C100F157C127
:100E300001F158C102F159C103F1F3EC0CF003BF09
:100E400069EF07F00E0EDEEC04F0E8CF0CF10F0EA8
:100E5000DEEC04F0E8CF0DF1100EDEEC04F0E8CF8C
:100E60000EF1110EDEEC04F0E8CF0FF128EC0CF0DF
:100E700056C104F157C105F158C106F159C107F136
:100E8000F3EC0CF00782ECEC0BF028EC0CF0079282
:100E9000ECEC0BF056C100F157C101F158C102F161
:100EA00059C103F10792ECEC0BF0E10E046F9E0EBA
:100EB000056F3C0E066F050E076FF3EC0CF000C1DA
:100EC0000CF101C10DF102C10EF103C10FF1A2EF4E
:100ED00007F00101800E006F1A0E016F060E026FFF
:100EE000000E036F42C104F143C105F144C106F194
:100EF00045C107F1F3EC0CF003AF83EF07F0C7EC4B
:100F00000DF0B5EF07F00E0EDEEC04F0E8CF0CF1BB
:100F10000F0EDEEC04F0E8CF0DF1100EDEEC04F065
:100F2000E8CF0EF1110EDEEC04F0E8CF0FF142C174
:100F300000F143C101F144C102F145C103F107824F
:100F4000ECEC0BF00CC100F10DC101F10EC102F18E
:100F50000FC103F10101000E046F000E056F010EB9
:100F6000066F000E076F21EC0DF08DEC0DF01D6784
:100F7000BFEF07F00401200E826FC2EF07F00401FB
:100F80002D0E826F60EC05F024C182F40401300E56
:100F9000822760EC05F025C182F40401300E82271F
:100FA00060EC05F004012E0E826F60EC05F026C1A6
:100FB00082F40401300E822760EC05F027C182F430
:100FC0000401300E822760EC05F004016D0E826F83
:100FD00060EC05F004012C0E826F60EC05F042C15C
:100FE00000F143C101F144C102F145C103F1010126
:100FF0008DEC0DF01EC182F40401300E822760ECEE
:1010000005F01FC182F40401300E822760EC05F068
:1010100020C182F40401300E822760EC05F021C16A
:1010200082F40401300E822760EC05F022C182F4C4
:101030000401300E822760EC05F023C182F4040124
:10104000300E822760EC05F024C182F40401300EDA
:10105000822760EC05F025C182F40401300E82275E
:1010600060EC05F026C182F40401300E822760ECAA
:1010700005F027C182F40401300E822760EC05F0F0
:101080000401480E826F60EC05F004017A0E826F55
:1010900060EC05F004012C0E826F60EC05F056C187
:1010A00000F157C101F158C102F159C103F1010129
:1010B0008DEC0DF01EC182F40401300E822760EC2D
:1010C00005F01FC182F40401300E822760EC05F0A8
:1010D00020C182F40401300E822760EC05F021C1AA
:1010E00082F40401300E822760EC05F022C182F404
:1010F0000401300E822760EC05F023C182F4040164
:10110000300E822760EC05F024C182F40401300E19
:10111000822760EC05F025C182F40401300E82279D
:1011200060EC05F026C182F40401300E822760ECE9
:1011300005F027C182F40401300E822760EC05F02F
:101140000401630E826F60EC05F004012C0E826FC7
:1011500060EC05F0078452C100F153C101F154C1A4
:1011600002F155C103F1079401010A0E046F000E4C
:10117000056F000E066F000E076F02EC0DF0000EFB
:10118000046F120E056F000E066F000E076F21EC44
:101190000DF08DEC0DF01EC182F40401300E82279B
:1011A00060EC05F01FC182F40401300E822760EC70
:1011B00005F020C182F40401300E822760EC05F0B6
:1011C00021C182F40401300E822760EC05F022C1B7
:1011D00082F40401300E822760EC05F023C182F412
:1011E0000401300E822760EC05F024C182F4040172
:1011F000300E822760EC05F004012E0E826F60EC49
:1012000005F025C182F40401300E822760EC05F060
:1012100026C182F40401300E822760EC05F027C15C
:1012200082F40401300E822760EC05F00401730E95
:10123000826F60EC05F004012C0E826F60EC05F00B
:10124000C7EC0DF04CC100F14DC101F18AEC0AF080
:101250006AEC05F061EF09F00401630E826F60EC47
:1012600005F004012C0E826F60EC05F066EC09F0CD
:1012700004012C0E826F60EC05F0D9EC09F004013A
:101280002C0E826F60EC05F055EC0AF004012C0E78
:10129000826F60EC05F00101F80E006FCD0E016F5A
:1012A000660E026F030E036F7BEC09F004012C0E37
:1012B000826F60EC05F06BEC0AF06AEC05F061EF10
:1012C00009F003018A6B0790EAEF0AF0D8900E0E3E
:1012D000DEEC04F0E8CF00F10F0EDEEC04F0E8CF16
:1012E00001F1100EDEEC04F0E8CF02F1110EDEEC9D
:1012F00004F0E8CF03F10101000E046F000E056F4A
:10130000010E066F000E076F21EC0DF08DEC0DF055
:101310001EC182F40401300E822760EC05F01FC16B
:1013200082F40401300E822760EC05F020C182F4C3
:101330000401300E822760EC05F021C182F4040123
:10134000300E822760EC05F022C182F40401300ED9
:10135000822760EC05F023C182F40401300E82275D
:1013600060EC05F024C182F40401300E822760ECA9
:1013700005F025C182F40401300E822760EC05F0EF
:1013800004012E0E826F60EC05F026C182F4040188
:10139000300E822760EC05F027C182F40401300E84
:1013A000822760EC05F004016D0E826F60EC05F0A1
:1013B0001200120EDEEC04F0E8CF00F1130EDEECAA
:1013C00004F0E8CF01F1140EDEEC04F0E8CF02F1F6
:1013D000150EDEEC04F0E8CF03F101010A0E046FF4
:1013E000000E056F000E066F000E076F02EC0DF089
:1013F000000E046F120E056F000E066F000E076FD1
:1014000021EC0DF08DEC0DF01EC182F40401300EC4
:10141000822760EC05F01FC182F40401300E8227A0
:1014200060EC05F020C182F40401300E822760ECEC
:1014300005F021C182F40401300E822760EC05F032
:1014400022C182F40401300E822760EC05F023C132
:1014500082F40401300E822760EC05F024C182F48E
:101460000401300E822760EC05F004012E0E826F1D
:1014700060EC05F025C182F40401300E822760EC97
:1014800005F026C182F40401300E822760EC05F0DD
:1014900027C182F40401300E822760EC05F00401BC
:1014A000730E826F60EC05F012000A0EDEEC04F0A1
:1014B000E8CF00F10B0EDEEC04F0E8CF01F10C0EEA
:1014C000DEEC04F0E8CF02F10D0EDEEC04F0E8CF24
:1014D00003F18AEF0AF0060EDEEC04F0E8CF00F12B
:1014E000070EDEEC04F0E8CF01F1080EDEEC04F0AC
:1014F000E8CF02F1090EDEEC04F0E8CF03F18AEF49
:101500000AF00101C7EC0DF007844AC100F14BC19C
:1015100001F107940101E80E046F800E056F000EC3
:10152000066F000E076F02EC0DF0000E046F040E44
:10153000056F000E066F000E076F21EC0DF0880E90
:10154000046F130E056F000E066F000E076FF3ECAD
:101550000CF00A0E046F000E056F000E066F000EF1
:10156000076F21EC0DF08DEC0DF001011D67BEEF52
:101570000AF00401200E826FC1EF0AF004012D0E63
:10158000826F60EC05F024C182F40401300E8227E2
:1015900060EC05F025C182F40401300E822760EC76
:1015A00005F026C182F40401300E822760EC05F0BC
:1015B00004012E0E826F60EC05F027C182F4040155
:1015C000300E822760EC05F00401430E826F60EC60
:1015D00005F0120081A8A8EF0BF007A861EF0BF04F
:1015E0000101800E006F1A0E016F060E026F000ED1
:1015F000036F3EC104F13FC105F140C106F141C195
:1016000007F1F3EC0CF003BFA8EF0BF0E6EC0BF0E6
:101610003EC100F13FC101F140C102F141C103F1FE
:101620000782ECEC0BF00CC104F10DC105F10EC109
:1016300006F10FC107F1F80E006FCD0E016F660EB7
:10164000026F030E036FF3EC0CF00E0E0C6E00C174
:101650000BF0C8EC04F00F0E0C6E01C10BF0C8ECDF
:1016600004F0100E0C6E02C10BF0C8EC04F0110E69
:101670000C6E03C10BF0C8EC04F007840101C7EC49
:101680000DF04AC100F14BC101F107940A0E0C6E36
:1016900000C10BF0C8EC04F00B0E0C6E01C10BF096
:1016A000C8EC04F00C0E0C6E02C10BF0C8EC04F098
:1016B0000D0E0C6E03C10BF0C8EC04F00798A8EFF8
:1016C0000BF007AAA8EF0BF007840101C7EC0DF09F
:1016D0004AC100F14BC101F10794060E0C6E00C126
:1016E0000BF0C8EC04F0070E0C6E01C10BF0C8EC57
:1016F00004F0080E0C6E02C10BF0C8EC04F0090EE9
:101700000C6E03C10BF0C8EC04F0078452C100F169
:1017100053C101F154C102F155C103F10794120EF6
:101720000C6E00C10BF0C8EC04F0130E0C6E01C17E
:101730000BF0C8EC04F0140E0C6E02C10BF0C8ECF8
:1017400004F0150E0C6E03C10BF0C8EC04F0079A00
:101750000401805181197F0B0BE09EA809D014EE83
:1017600000F081517F0BE126E750812B0F01AD6E18
:1017700026EF05F00CC100F10DC101F10EC102F11F
:101780000FC103F1000E046F000E056F010E066F0E
:10179000000E076F21EC0DF01DA1E5EF0BF01451C9
:1017A000D8B4E5EF0BF00CC100F10DC101F10EC191
:1017B00002F10FC103F1000E046F000E056F0A0E57
:1017C000066F000E076F21EC0DF0120001010C6B8B
:1017D0000D6B0E6B0F6B12000101005305E10153FD
:1017E00003E1025301E1002BC3EC0CF0C7EC0DF058
:1017F0002C51006F2D51016F420E046F4B0E056F7F
:10180000000E066F000E076F02EC0DF000C104F130
:1018100001C105F102C106F103C107F10CC100F1DC
:101820000DC101F10EC102F10FC103F107B21DEFAD
:101830000CF0F7EC0CF01FEF0CF0F3EC0CF000C127
:101840000CF101C10DF102C10EF103C10FF1120043
:10185000C7EC0DF04CC100F14DC101F1210E046F38
:10186000000E056F000E066F000E076F02EC0DF004
:10187000320E046F000E056F000E066F000E076F2C
:1018800021EC0DF0060EDEEC04F0E8CF04F1070EBB
:10189000DEEC04F0E8CF05F1080EDEEC04F0E8CF52
:1018A00006F1090EDEEC04F0E8CF07F1F3EC0CF0E2
:1018B00000C118F101C119F102C11AF103C11BF1F4
:1018C000290E046F000E056F000E066F000E076FE5
:1018D00002EC0DF0EE0E046F430E056F000E066F66
:1018E000000E076FF7EC0CF018C104F119C105F1F7
:1018F0001AC106F11BC107F102EC0DF000C110F195
:1019000001C111F102C112F103C113F1120EDEEC9B
:1019100004F0E8CF04F1130EDEEC04F0E8CF05F19B
:10192000140EDEEC04F0E8CF06F1150EDEEC04F048
:10193000E8CF07F10D0E006F000E016F000E026F71
:10194000000E036F02EC0DF0180E046F000E056F11
:10195000000E066F000E076F21EC0DF010C104F1B0
:1019600011C105F112C106F113C107F1F7EC0CF03A
:101970006A0E046F2A0E056F000E066F000E076FC9
:10198000F3EC0CF01200BF0EFA6E200E2D6F2C6BD4
:10199000D8900037013702370337D8B0D4EF0CF0B6
:1019A0002D2FC9EF0CF02C072D070353D8B41200CC
:1019B0000331070B8009326F03390F0B010F2C6FB6
:1019C00080EC5FF0336F2C0580EC5FF0335D335FAC
:1019D0002C6B3233D8B02C272C3332A9E9EF0CF022
:1019E00033512C271200ECEC0DF0D8B0120003514B
:1019F0000719286FAFEC0DF0D8900751031928AFE5
:101A0000800F1200286BD3EC0DF0D8A0E9EC0DF09C
:101A1000D8B01200BEEC0DF0C7EC0DF01F0E296F10
:101A2000FFEC0DF00B35D8B0AFEC0DF0D8A00335BE
:101A3000D8B01200292F10EF0DF028B1D6EC0DF020
:101A40001200286B04510511061107110008D8A0D7
:101A5000D3EC0DF0D8A0E9EC0DF0D8B01200086B73
:101A6000096B0A6B0B6BFFEC0DF01F0E296FFFEC7F
:101A70000DF007510B5DD8A44AEF0DF006510A5D39
:101A8000D8A44AEF0DF00551095DD8A44AEF0DF036
:101A90000451085DD8A05DEF0DF00451085F0551B9
:101AA000D8A0053D095F0651D8A0063D0A5F075141
:101AB000D8A0073D0B5FD8900081292F37EF0DF09C
:101AC00028B1D6EC0DF0286BD3EC0DF0D89003ECD8
:101AD0000EF007510B5DD8A47AEF0DF006510A5DA8
:101AE000D8A47AEF0DF00551095DD8A47AEF0DF076
:101AF0000451085DD8A089EF0DF0003F89EF0DF08B
:101B0000013F89EF0DF0023F89EF0DF0032BD8B4B0
:101B1000120028B1D6EC0DF012000101286BD3ECB5
:101B20000DF0D8B0120008EC0EF0200E296F00372F
:101B300001370237033711EE27F00A0E2A6FE73616
:101B40000A0EE75CD8B0E76EE5522A2F9FEF0DF042
:101B5000292F97EF0DF028B11D81D8901200045164
:101B600000270551D8B0053D01270651D8B0063DE4
:101B700002270751D8B0073D032712000051086F14
:101B80000151096F02510A6F03510B6F12000101DD
:101B9000006B016B026B036B12000101046B056BA0
:101BA000066B076B12000335D8A012000351800B9F
:101BB000001F011F021F031F003FE6EF0DF0013F52
:101BC000E6EF0DF0023FE6EF0DF0032B282B032587
:101BD00012000735D8A012000751800B041F051F03
:101BE000061F071F043FFCEF0DF0053FFCEF0DF053
:101BF000063FFCEF0DF0072B282B072512000037BE
:101C0000013702370337083709370A370B37120015
:101C10001D6B1E6B1F6B206B216B226B236B246B68
:081C2000256B266B276B1200F7
:10BF0000E844F926000C160C2B0C3F0C520C640C68
:10BF1000760C860C960CA50CB30CC10CCF0CDC0C6B
:06BF2000E80CF40C000C1B
:00000001FF
